:100000000C9462010C9497110C94C4110C948A0105
:100010000C948A010C948A010C948A010C948A0134
:100020000C948A010C948A010C948A010C948A0124
:100030000C948A010C948A010C948A010C948A0114
:100040000C9421150C948A010C94D8120C9426134C
:100050000C948A010C948A010C948A010C948A01F4
:100060000C948A010C948A01000021104220633014
:100070008440A550C660E770088129914AA16BB100
:100080008CC1ADD1CEE1EFF13112100273325222A8
:10009000B5529442F772D662399318837BB35AA350
:1000A000BDD39CC3FFF3DEE3622443342004011478
:1000B000E664C774A44485546AA54BB528850995A0
:1000C000EEE5CFF5ACC58DD5533672261116300648
:1000D000D776F6669556B4465BB77AA719973887F0
:1000E000DFF7FEE79DD7BCC7C448E5588668A77808
:1000F0004008611802282338CCC9EDD98EE9AFF940
:10010000488969990AA92BB9F55AD44AB77A966AE7
:10011000711A500A333A122AFDDBDCCBBFFB9EEB8F
:10012000799B588B3BBB1AABA66C877CE44CC55CB7
:10013000222C033C600C411CAEED8FFDECCDCDDDDF
:100140002AAD0BBD688D499D977EB66ED55EF44E87
:10015000133E322E511E700E9FFFBEEFDDDFFCCF2F
:100160001BBF3AAF599F788F8891A981CAB1EBA183
:100170000CD12DC14EF16FE18010A100C230E320FF
:100180000450254046706760B9839893FBA3DAB3A7
:100190003DC31CD37FE35EF3B1029012F322D2324F
:1001A0003542145277625672EAB5CBA5A895898577
:1001B0006EF54FE52CD50DC5E234C324A01481049F
:1001C0006674476424540544DBA7FAB79987B89747
:1001D0005FE77EF71DC73CD7D326F2369106B016EF
:1001E00057667676154634564CD96DC90EF92FE907
:1001F000C899E9898AB9ABA944586548067827683F
:10020000C018E1088238A3287DCB5CDB3FEB1EFBE6
:10021000F98BD89BBBAB9ABB754A545A376A167A8E
:10022000F10AD01AB32A923A2EFD0FED6CDD4DCDB6
:10023000AABD8BADE89DC98D267C076C645C454CDE
:10024000A23C832CE01CC10C1FEF3EFF5DCF7CDF86
:100250009BAFBABFD98FF89F176E367E554E745E2E
:10026000932EB23ED10EF01E0000000024002700A5
:100270002A0000000000250028002B0000000000DC
:1002800023002600290004040404040404040202D8
:100290000202020203030303030301020408102005
:1002A0004080010204081020010204081020000010
:1002B0000007000201000003040600000000000027
:1002C0000000921411241FBECFEFD8E0DEBFCDBFD7
:1002D00011E0A0E0B1E0EAEEFBE202C005900D9271
:1002E000A631B107D9F718E0A6E1B1E001C01D922F
:1002F000A730B107E1F712E0C4ECD2E004C02297C6
:10030000FE010E94EF15C23CD107C9F70E94E81414
:100310000C94F3150C94000061E070E040E050E0B4
:1003200016C0342F2227FB01E858F94F8081E82FAF
:10033000F0E0852F9927E827F927EE0FFF1FE859EE
:10034000FF4F45915491422753276F5F7F4F809114
:10035000B0069091B106861797071CF74093CA061E
:100360005093CB06E091B006F091B106E658F94FF4
:100370004083E091B006F091B106E758F94F508301
:100380008091B0069091B10602969093B106809349
:10039000B0060895AF92BF92CF92DF92EF92FF9294
:1003A0000F931F93CF93DF9310920D0610920C06BC
:1003B0008FEF8093100610920F0610920E068AEEB1
:1003C0008093460286EA809347021092480284E0B6
:1003D00090E090939D0580939C0583E090E090933E
:1003E0009F0580939E0540E050E0C1E0D0E031E001
:1003F000E32EF12C012D112D10920F0610920E06F6
:10040000BE01042E02C0660F771F0A94E2F766C091
:1004100080910E0690910F06FC01EE0FFF1FE80F72
:10042000F91FE854FA4F808190E086239723892BA7
:10043000B9F0E0919E05F0919F05EB5BFD4F2081A7
:1004400080919C0590919D055701680104C0AA0CFC
:10045000BB1CCC1CDD1C8A95D2F72A29208319C02D
:10046000E0919E05F0919F05EB5BFD4F208180910F
:100470009C0590919D055701680104C0AA0CBB1C06
:10048000CC1CDD1C8A95D2F7D601C501809582234C
:10049000808380919C0590919D05019690939D0588
:1004A00080939C0580919C0590919D0508976CF028
:1004B00010929D0510929C0580919E0590919F053C
:1004C000019690939F0580939E0580910E069091D2
:1004D0000F06019690930F0680930E0680910E06EC
:1004E00090910F064C970CF493CF4F5F5F4F4830BD
:1004F000510509F081CF40E050E0C1E0D0E0B1E02B
:10050000EB2EF12C012D112D10920F0610920E06DC
:10051000BE01042E02C0660F771F0A94E2F766C080
:1005200080910E0690910F06FC01EE0FFF1FE80F61
:10053000F91FE854FA4F818190E086239723892B95
:10054000B9F0E0919E05F0919F05EB5BFD4F208196
:1005500080919C0590919D055701680104C0AA0CEB
:10056000BB1CCC1CDD1C8A95D2F72A29208319C01C
:10057000E0919E05F0919F05EB5BFD4F20818091FE
:100580009C0590919D055701680104C0AA0CBB1CF5
:10059000CC1CDD1C8A95D2F7D601C501809582233B
:1005A000808380919C0590919D05019690939D0577
:1005B00080939C0580919C0590919D0508976CF017
:1005C00010929D0510929C0580919E0590919F052B
:1005D000019690939F0580939E0580910E069091C1
:1005E0000F06019690930F0680930E0680910E06DB
:1005F00090910F064C970CF493CF4F5F5F4F4430B0
:10060000510509F081CF44E050E0C1E0D0E031E095
:10061000E32EF12C012D112D10920F0610920E06D3
:10062000BE01042E02C0660F771F0A94E2F766C06F
:1006300080910E0690910F06FC01EE0FFF1FE80F50
:10064000F91FE854FA4F818190E086239723892B84
:10065000B9F0E0919E05F0919F05EB5BFD4F208185
:1006600080919C0590919D055701680104C0AA0CDA
:10067000BB1CCC1CDD1C8A95D2F72A29208319C00B
:10068000E0919E05F0919F05EB5BFD4F20818091ED
:100690009C0590919D055701680104C0AA0CBB1CE4
:1006A000CC1CDD1C8A95D2F7D601C501809582232A
:1006B000808380919C0590919D05019690939D0566
:1006C00080939C0580919C0590919D0508976CF006
:1006D00010929D0510929C0580919E0590919F051A
:1006E000019690939F0580939E0580910E069091B0
:1006F0000F06019690930F0680930E0680910E06CA
:1007000090910F064B970CF493CF4F5F5F4F48309B
:10071000510509F081CF40E050E0C1E0D0E0B1E008
:10072000EB2EF12C012D112D10920F0610920E06BA
:10073000BE01042E02C0660F771F0A94E2F766C05E
:1007400080910E0690910F06FC01EE0FFF1FE80F3F
:10075000F91FE854FA4F828190E086239723892B72
:10076000B9F0E0919E05F0919F05EB5BFD4F208174
:1007700080919C0590919D055701680104C0AA0CC9
:10078000BB1CCC1CDD1C8A95D2F72A29208319C0FA
:10079000E0919E05F0919F05EB5BFD4F20818091DC
:1007A0009C0590919D055701680104C0AA0CBB1CD3
:1007B000CC1CDD1C8A95D2F7D601C5018095822319
:1007C000808380919C0590919D05019690939D0555
:1007D00080939C0580919C0590919D0508976CF0F5
:1007E00010929D0510929C0580919E0590919F0509
:1007F000019690939F0580939E0580910E0690919F
:100800000F06019690930F0680930E0680910E06B8
:1008100090910F064B970CF493CF4F5F5F4F48308A
:10082000510509F081CF84E090E090939D0580937D
:100830009C0583E090E090939F0580939E0581E066
:1008400090E090930F0680930E0641E0E42EF12C89
:10085000012D112D8EC080911006880F80931006F7
:10086000809110062091100690E034E095958795D0
:100870003A95E1F781709070221F2227221F30E005
:100880008217930721F080911006816003C0809148
:1008900010068E7F8093100620911006E0919E0531
:1008A000F0919F05EB5BFD4F808140919C0550913D
:1008B0009D0590E002C0959587954A95E2F730E056
:1008C0008227932780FF17C0E0919E05F0919F0536
:1008D000EB5BFD4F208180919C0590919D05B801B7
:1008E000A70104C0440F551F661F771F8A95D2F7D2
:1008F000242B208319C0E0919E05F0919F05EB5BAE
:10090000FD4F208180919C0590919D0557016801C4
:1009100004C0AA0CBB1CCC1CDD1C8A95D2F7D601E6
:10092000C50180958223808380919C0590919D05CF
:10093000019690939D0580939C0580919C059091D4
:100940009D0508976CF010929D0510929C05809172
:100950009E0590919F05019690939F0580939E051B
:1009600080910E0690910F06019690930F0680934A
:100970000E0680910E0690910F06855992400CF458
:100980006ACFDF91CF911F910F91FF90EF90DF9091
:10099000CF90BF90AF90089540911006209110061F
:1009A0008091100630E03595279550E04227532777
:1009B0004170507090E095958795959587958170D9
:1009C00090704817590709F180910D0620910C0687
:1009D00090E0FC01EE0FFF1FE80FF91FE20FF11D81
:1009E000E854FA4F408120910E0630910F0681E0C5
:1009F00090E0A0E0B0E004C0880F991FAA1FBB1FC1
:100A00002A95D2F7482B408321C080910D06209172
:100A10000C0690E0FC01EE0FFF1FE80FF91FE20F3C
:100A2000F11DE854FA4F408120910E0630910F06D7
:100A300081E090E0A0E0B0E004C0880F991FAA1FF9
:100A4000BB1F2A95D2F780958423808380910E0660
:100A500090910F06019690930F0680930E062091B9
:100A600010068091100690E095958795959587954D
:100A700030E08227932780FF21C080910D062091CE
:100A80000C0690E0FC01EE0FFF1FE80FF91FE20FCC
:100A9000F11DE854FA4F408120910E0630910F0667
:100AA00081E090E0A0E0B0E004C0880F991FAA1F89
:100AB000BB1F2A95D2F7482B408321C080910D0699
:100AC00020910C0690E0FC01EE0FFF1FE80FF91FCC
:100AD000E20FF11DE854FA4F408120910E0630914B
:100AE0000F0681E090E0A0E0B0E004C0880F991FFD
:100AF000AA1FBB1F2A95D2F78095842380838091FB
:100B00000E0690910F06019690930F0680930E06A5
:100B10000895CF93DF9310920D0610920C06109259
:100B2000100610920F0610920E0681E090E045C06C
:100B3000C0E0D0E080911006880F80931006E0910D
:100B40003C06F0913D06EF5EF94F808190E00C2E5F
:100B500002C0959587950A94E2F780FF04C08091C2
:100B60001006816003C0809110068E7F809310066E
:100B70000E94CC0480910E0690910F060897A4F075
:100B800010920F0610920E0680910C068F5F8093D4
:100B90000C0680910C06833038F010920C06809180
:100BA0000D068F5F80930D062196C830D10511F692
:100BB00080913C0690913D06019690933D0680936E
:100BC0003C0680913C0690913D068A970CF4B0CF8C
:100BD00080911006880F80931006809110068E7FFA
:100BE000809310060E94CC0480911006880F809399
:100BF0001006809110068E7F809310060E94CC0410
:100C0000DF91CF9108958091100683FFC6C0809137
:100C1000100686FFC2C004C08091100686FDC1C0C8
:100C200080911006880F80931006809110068E7FA9
:100C3000809310068091AA0580FFBCC080911006A9
:100C400080FFB8C004C08091100680FDB7C08091BD
:100C50000D0620910C0690E0FC01EE0FFF1FE80F3F
:100C6000F91FE20FF11DE854FA4F408120910E0662
:100C700030910F0681E090E0A0E0B0E004C0880F62
:100C8000991FAA1FBB1F2A95D2F7809584238083C2
:100C900080910D068F5F80930D0680910C0688234E
:100CA00001F580910D068C31E0F010920D068091D7
:100CB0000E0690910F06019790930F0680930E06F3
:100CC00080910E0690910F0697FF0BC087E090E091
:100CD00090930F0680930E0680910C068F5F809391
:100CE0000C0680910C06813079F480910D068C31D0
:100CF00058F010920D0680910E0690910F06019704
:100D000090930F0680930E0680910C068130A9F413
:100D100080910D068B3189F480910E0690910F061B
:100D200004975CF410920D0680910E0690910F06C8
:100D3000019790930F0680930E0680910E06909176
:100D40000F0697FF0BC087E090E090930F0680930B
:100D50000E0680910C068F5F80930C0680910C0626
:100D6000823009F04CC080910D068B3108F447C0E9
:100D700010920D0680910E0690910F0601979093A8
:100D80000F0680930E0680910E0690910F0697FF36
:100D900036C083E08093B50608958091100683FFE6
:100DA0003BCF80911006880F80931006809110062B
:100DB00081603ECF8091AA0580FF45CF80910D06CE
:100DC00020910C0690E0FC01EE0FFF1FE80FF91FC9
:100DD000E20FF11DE854FA4F408120910E06309148
:100DE0000F0681E090E0A0E0B0E004C0880F991FFA
:100DF000AA1FBB1F2A95D2F7482B408349CF0895DD
:100E00008091100687FF19C08091100682FF15C0DF
:100E100004C08091100682FD14C0809110068E7F60
:100E20008093100680913B0690E09595879580937E
:100E30003B0680913B068F7713C08091100687FF99
:100E4000E8CF8091100681608093100680913B0668
:100E500090E09595879580933B0680913B0680684E
:100E600080933B0680911006880F809310060895AA
:100E70008091B7058F5F8093B7058091B705883063
:100E800000F11092B705E0910201F0910301E95ED3
:100E9000FE4F80818093A005809102019091030113
:100EA0000197909303018093020180910201909138
:100EB0000301892B31F48CE291E09093030180933C
:100EC0000201E6E1F0E0DF01A056BA4F8C9190E01C
:100ED000959587958C939F0121503040F901E056FC
:100EE000FA4F808180FF03C08C91806802C08C9192
:100EF0008F778C938FEF2F3F380711F0F901E3CFF5
:100F000008958091CC069091CD0601969093CD06E0
:100F10008093CC068091BB06882331F485E00E9443
:100F20008412892B51F005C085E00E948412892B20
:100F300021F480911601806803C0809116018F779B
:100F400080931601809144028F5F809344028091C8
:100F50004402883009F5E0910001F091010180918F
:100F60001601E95EFE4F808380910001909101019E
:100F7000019790930101809300018091000190916D
:100F80000101892B31F48CE291E09093010180936F
:100F900000011092440207C08091160190E09595DF
:100FA00087958093160181E08093B706089580911C
:100FB000CC069091CD0601969093CD068093CC06F9
:100FC0008091C1069091C20601979093C2068093CA
:100FD000C1068091B806843021F08091B806853032
:100FE00059F51092C8061092C7068091C906815023
:100FF0008093C90686E00E948412019719F486E066
:1010000060E002C086E061E00E9430128091B80684
:10101000853091F48091BC06882331F486E00E94EB
:101020008412019749F405C086E00E948412892B3E
:1010300019F486E08093B8068091B806873029F0CD
:101040008091B806883009F079C08091C7069091E8
:10105000C80601969093C8068093C7068091C7067C
:101060009091C806803691055CF01092C8061092E7
:10107000C7068091C6068F5F8093C6068091C6061C
:10108000E0919A05F0919B05EB5BFD4F80812091EB
:101090009C0530919D0590E002C0959587952A9515
:1010A000E2F780FF05C08091BC06813029F407C0BB
:1010B0008091BC06813019F486E061E002C086E0D0
:1010C00060E00E94301280919C0590919D050196F0
:1010D00090939D0580939C0580919C0590919D0522
:1010E0000897D1F410929D0510929C0580919A0565
:1010F00090919B05019690939B0580939A05809112
:101100009A0590919B058355934034F081E090E0DF
:1011100090939B0580939A058091B806883071F46E
:10112000209198053091990580919A0590919B05A1
:101130002817390719F489E08093B80681E0809375
:10114000BA0608958091AE058A3AC1F48091AD0542
:101150008A3AA1F48091AC058A3A81F48091AB057A
:101160008A3A61F481E08093B5068091C40681607B
:101170008093C40689E060E00E9430120895809157
:10118000C40682608093C40688E061E00E94301249
:101190008091BF0625E0829FC00111249093C20672
:1011A0008093C1064091C1065091C2068091C0064D
:1011B00090E02BEF34E0BC01629FC001639F900D73
:1011C000729F900D1124840F951F9093C2068093F7
:1011D000C10682E08093B8068093B6061092C606D8
:1011E0001092C50608958091C4068D7F8093C40631
:1011F00088E060E00E94301281E08093B80610928F
:10120000B9068093B6060895CF93DF9380ED80935F
:1012100079060E948C01C1E0D0E009C0FE01E858C7
:10122000F94F60818CED97E00E94521421968091D5
:10123000B0069091B1068C179D0784F7DF91CF918E
:101240000895FF920F931F938091AE058A3A09F09B
:1012500050C08091AD058A3A09F04BC08091AC0531
:101260008E3609F046C08091AB058A3009F041C046
:1012700082E08093B50610920C0610920D0687E06E
:1012800090E090930F0680930E068FEF80931006E8
:101290001092B406809104018F5F80930401F3E003
:1012A000FF2EF0927A0610927B0685E180937C06F1
:1012B00010927D0610927E0606E010E01093B106B3
:1012C0000093B0060E940409F0927A0610927B0601
:1012D00086E180937C068091040180937D06809155
:1012E000B40680937E061093B1060093B0060E9468
:1012F00004091F910F91FF90089510920D0610920E
:101300000C061092100610923D0610923C0614C175
:1013100010923B0680910D0690E020910C06FC0196
:10132000EE0FFF1FE80FF91FE20FF11DE854FA4F0F
:10133000808186FF04C080911006806803C0809180
:1013400010068F77809310060E94000780910D068B
:1013500090E020910C06FC01EE0FFF1FE80FF91F33
:10136000E20FF11DE854FA4F808184FF04C08091A0
:101370001006806803C0809110068F778093100656
:101380000E94000780910D0690E020910C06FC0160
:10139000EE0FFF1FE80FF91FE20FF11DE854FA4F9F
:1013A000808182FF04C080911006806803C0809114
:1013B00010068F77809310060E94000780910D061B
:1013C00090E020910C06FC01EE0FFF1FE80FF91FC3
:1013D000E20FF11DE854FA4F808180FF04C0809134
:1013E0001006806803C0809110068F7780931006E6
:1013F0000E94000780910C068F5F80930C068091FD
:101400000C06833038F010920C0680910D068F5F29
:1014100080930D0680910D0690E020910C06FC0152
:10142000EE0FFF1FE80FF91FE20FF11DE854FA4F0E
:10143000808186FF04C080911006806803C080917F
:1014400010068F77809310060E94000780910D068A
:1014500090E020910C06FC01EE0FFF1FE80FF91F32
:10146000E20FF11DE854FA4F808184FF04C080919F
:101470001006806803C0809110068F778093100655
:101480000E94000780910D0690E020910C06FC015F
:10149000EE0FFF1FE80FF91FE20FF11DE854FA4F9E
:1014A000808182FF04C080911006806803C0809113
:1014B00010068F77809310060E94000780910D061A
:1014C00090E020910C06FC01EE0FFF1FE80FF91FC2
:1014D000E20FF11DE854FA4F808180FF04C0809133
:1014E0001006806803C0809110068F7780931006E5
:1014F0000E94000780910C068F5F80930C068091FC
:101500000C06833038F010920C0680910D068F5F28
:1015100080930D06E0913C06F0913D0680913B06DC
:10152000EF5EF94F808380913C0690913D060196D5
:1015300090933D0680933C0680913C0690913D0639
:1015400089970CF4E5CE84E08093B5068FE2809312
:101550007A0610927B0687E180937C0680910401D5
:1015600080937D068091B40680937E0610927F065C
:101570001092800610923D0610923C0617C0A09172
:101580003C06B0913D06E0913C06F0913D06EF5ED1
:10159000F94F8081AF57B94F8C9380913C06909161
:1015A0003D06019690933D0680933C0680913C0653
:1015B00090913D0689971CF382E390E09093B106E9
:1015C0008093B0060E9404090895209141062131BC
:1015D00009F040C020937A0610927B0681E980933F
:1015E0007C0691E390937D0620937E0684E48093AD
:1015F0007F0686E5809380068DE2809381068DE4E8
:101600008093820685E48093830687E48093840632
:1016100021E42093850680E28093860682E580930C
:101620008706909388068EE28093890690938A06B7
:1016300083E380938B0620938C0684E190E0909363
:10164000B1068093B0060E94040981E08093B80639
:101650008093B606809141068231E1F485E0809363
:101660007A0610927B0682E980937C0683E1809360
:101670007D0689E080937E0680E180937F0681E08D
:101680008093800688E090E09093B1068093B00646
:101690000E94040980914106843109F054C0809170
:1016A0004206803CE9F5809144068093BD06809116
:1016B00045068093BE06809146068093BF068091C2
:1016C00047068093C0068091BD0680FF04C081E07C
:1016D0008093BB0602C01092BB068091BD0681FFBD
:1016E00004C081E08093BC0602C01092BC068091C9
:1016F000BD0682FF03C01092CE0603C081E0809336
:10170000CE068091BD0682FF03C01092CF0603C0B3
:1017100081E08093CF0681E08093CE068093CF0650
:1017200082E080937A0610927B0684E980937C069F
:1017300086E080937D0685E090E09093B1068093EB
:10174000B0060E940409809141068031D1F4909145
:101750003F069230B1F4809142068093C306909385
:101760007A0610927B0680E980937C0686E080935F
:101770007D0685E090E09093B1068093B0060E94CC
:10178000040980914106803169F580913F068130DE
:1017900049F588E080937A0610927B0680E9809371
:1017A0007C0687E480937D068091C40680937E0644
:1017B0008091B60680937F0685E1809380068CEF4A
:1017C000809381068091C506809382068091C6062B
:1017D000809383068BE090E09093B1068093B006EF
:1017E0000E94040980914106863181F48091BC06F3
:1017F000813019F486E061E002C086E060E00E947A
:1018000030120E94F30881E08093B906809141066E
:10181000873151F5809142068093040180914306FF
:101820008093B40621E030E0F901EB5BF94F808151
:10183000F901EF5EF94F80832F5F3F4F2A32310568
:1018400099F786E590E0909399058093980581E05B
:1018500090E090939B0580939A050E9489050E94D1
:10186000CA0182E08093B90680914106893199F5D9
:101870001092CD061092CC0628E030E041E050E016
:10188000E0919805F0919905D901A25CB94F8C912E
:10189000EB5BFD4F808380919805909199050196AF
:1018A000909399058093980580919805909199055A
:1018B0008355934024F050939905409398052F5FEA
:1018C0003F4F24313105E1F68091B906823019F499
:1018D00083E08093B906809141068A3109F04DC1B9
:1018E000809198059091990501979093990580931F
:1018F00098058091980590919905892B31F482E59E
:1019000093E0909399058093980580919805909124
:101910009905019790939905809398058091980572
:1019200090919905892B31F482E593E09093990584
:1019300080939805809198059091990501979093CF
:101940009905809398058091980590919905892B28
:1019500031F482E593E09093990580939805E091A6
:101960009805F0919905EB5BFD4F85E580838091AB
:101970009805909199050196909399058093980503
:1019800080919805909199058355934034F081E0BA
:1019900090E09093990580939805E0919805F091D7
:1019A0009905EB5BFD4F85E58083809198059091CB
:1019B00099050196909399058093980580919805D3
:1019C000909199058355934034F081E090E0909395
:1019D000990580939805E0919805F0919905EB5B46
:1019E000FD4F85E58083809198059091990501963A
:1019F0009093990580939805809198059091990509
:101A00008355934034F081E090E090939905809362
:101A10009805E0919805F0919905EB5BFD4F85E500
:101A200080838091980590919905019690939905EE
:101A300080939805809198059091990583559340DE
:101A400034F081E090E09093990580939805E091BF
:101A50009805F0919905EB5BFD4F88EC80838091B0
:101A60009805909199050196909399058093980512
:101A700080919805909199058355934034F081E0C9
:101A800090E09093990580939805E0919805F091E6
:101A90009905EB5BFD4F8AE78083809198059091D3
:101AA00099050196909399058093980580919805E2
:101AB000909199058355934034F081E090E09093A4
:101AC000990580939805E0919805F0919905EB5B55
:101AD000FD4F108280919805909199050196909301
:101AE0009905809398058091980590919905835563
:101AF000934034F081E090E09093990580939805AD
:101B0000E0919805F0919905EB5BFD4F1082809173
:101B10009805909199050196909399058093980561
:101B200080919805909199058355934034F081E018
:101B300090E09093990580939805E0919805F09135
:101B40009905EB5BFD4F1082809198059091990566
:101B500001969093990580939805809198059091AE
:101B600099058355934034F081E090E09093990576
:101B70008093980584E08093B906809141068F3167
:101B8000E1F590914206903CD1F486E080937A068C
:101B900010927B068FE980937C0690937D061092CD
:101BA0007E0610927F06109280061092810689E0D0
:101BB00090E09093B1068093B0060E940409909142
:101BC0004206913CD1F486E080937A0610927B061F
:101BD0008FE980937C0690937D0610927E0610928A
:101BE0007F06109280061092810689E090E0909323
:101BF000B1068093B0060E94040910923E0610922E
:101C00003F061092770610927606089583E180933E
:101C10007A0610927B0689E180937C06809104010C
:101C200080937D068091B40680937E0688EE809333
:101C30007F0683E08093800625E130E04EE150E0AE
:101C4000FA01E21BF30BD901A056BA4F8C91E85868
:101C5000F94F8083215030402930310589F71092A7
:101C60008D0610928E0686E190E09093B1068093E7
:101C7000B0060E940409089583E080937A061092CA
:101C80007B068AE180937C068091040180937D0627
:101C90008091B40680937E0686E090E09093B10632
:101CA0008093B0060E940409089580E061E877E01F
:101CB00043E050E00E94741181E067ED77E042E07C
:101CC00050E00E9474118091C4068E7F8093C406F8
:101CD0001092B7058AEF90E0909303018093020180
:101CE0008CE291E090930101809300011092B5067F
:101CF00089E061E00E9430121092B2061092B306A1
:101D000008950F931F93CF93DF938CED97E00E947C
:101D1000E813181619060CF500917606109177064F
:101D20008CED97E00E941914025C194FF801808332
:101D3000809176069091770601969093770680932E
:101D400076068091760690917706C89734F087E3FF
:101D500090E0909377068093760680913E06803DD2
:101D600021F0109277061092760680913E06803D13
:101D700099F4809176069091770605976CF0209102
:101D800076063091770680913F0690E004968217A0
:101D9000930714F40E94E50A8091BA06813009F095
:101DA00045C0209198053091990580919A059091B0
:101DB0009B058217930784F480919805909199056B
:101DC00020919A0530919B05821B930B6CE070E08B
:101DD0000E94A4156093C50620919805309199053D
:101DE00080919A0590919B052817390794F480916A
:101DF00098059091990520919A0530919B058E5AEE
:101E00009C4F821B930B6CE070E00E94A4156093C2
:101E1000C506209198053091990580919A05909179
:101E20009B052817390711F41092C5068091B80652
:101E3000882309F499C08091B806813031F48091EB
:101E4000B906882311F00E94BF088091B80682303D
:101E500049F48091C1069091C206059718F483E079
:101E60008093B8069091B806933061F48091B906DA
:101E7000823040F080E48093C90684E08093B80605
:101E80009093B6068091B806843039F48091C906E3
:101E9000823018F485E08093B8068091B8068630C9
:101EA00031F487E08093B80685E08093B606809190
:101EB000B806873009F045C08091CC069091CD06D8
:101EC000815C924110F00E94F3088091C506853034
:101ED000D0F480919A0590919B05CC9790939B05A7
:101EE00080939A0580919A0590919B051816190682
:101EF00054F080919A0590919B058E5A9C4F909337
:101F00009B0580939A058091C5068334D0F080911B
:101F1000980590919905CC97909399058093980591
:101F200080919805909199051816190654F08091A2
:101F30009805909199058E5A9C4F9093990580939E
:101F400098059091B806973049F48091B90684308D
:101F500029F488E08093B8069093B6068091B8067D
:101F6000893011F40E94F3088091B5068630C0F5DF
:101F700020910001309101018091020190910301B3
:101F80008217930794F480910201909103012091AC
:101F9000000130910101845D9E4F821B930B8B3FAA
:101FA00091051CF081E08093B706209102013091E9
:101FB000030180910001909101018217930784F43D
:101FC0008091020190910301209100013091010163
:101FD000821B930B8B3F91051CF081E08093B70629
:101FE0008091B706813009F02FC10E943807809197
:101FF000B506882331F48091B706813011F40E9430
:10200000A2088091B506813031F48091B706813005
:1020100011F40E9421098091B506823031F480913B
:10202000B706813011F40E9403068091B506833013
:1020300031F48091B706813011F40E947D098091BE
:10204000B506843039F48091B706813019F485E003
:102050008093B5068091B5068530D1F48091B7069E
:102060008130B1F405C00E9438078091B2068F5FBD
:102070008093B2068091B2068131A8F386E0809306
:10208000B5061092B20684E18093B3061092B706AB
:102090008091B506863009F0D7C08091B7068130AF
:1020A00009F0D2C08091B2068F5F8093B206809112
:1020B000B206823008F44FC08091B206893108F030
:1020C0004AC020910201309103018091000190915A
:1020D000010182179307CCF48091020190910301D2
:1020E0002091000130910101821B930B45976CF008
:1020F000C1E0D0E00E9438078091B2068F5F8093E4
:10210000B2062196C132D105A9F720910201309182
:102110000301809100019091010128173907DCF437
:102120008091020190910301209100013091010101
:10213000845D9E4F821B930B45976CF0C1E0D0E00D
:102140000E9438078091B2068F5F8093B206219675
:10215000C132D105A9F78091B2068934E1F48091AA
:10216000AC058535C1F48091AB058535A1F480912E
:10217000AA05853581F48091A905853561F48091A2
:10218000A805883C41F48091A7058A3721F40E9474
:10219000550E0E943C0E8091B3068431A1F48091CB
:1021A000B206823480F08091AB05853561F4809170
:1021B000AA058D3241F48091A905863121F410924F
:1021C000B7060E9438078091B306843111F58091DB
:1021D000B2068934F1F48091AC058535F1F5809132
:1021E000AB058D32D1F58091AA058631B1F511C0CC
:1021F0008091AB058D3221F08091AA05863191F551
:1022000085E58093AC058DE28093AB0586E18093F4
:10221000AA058091B206893431F48091B306809387
:10222000B4060E94060E8091B206803668F01092C5
:10223000B2068091B3068F5F8093B3068091B30698
:10224000853110F01092B3061092B7061092BA06BC
:10225000DF91CF911F910F9108958091AC05853545
:1022600039F6CECF0E94550E0E943C0ED2CF0F936E
:102270001F938DE061E00E94F11184E060E00E9414
:10228000F11185E060E00E94F11182E060E00E94BF
:10229000F11183E060E00E94F11186E061E00E94AC
:1022A000F11188E061E00E94F11189E061E00E9493
:1022B000F11188E060E00E94301289E061E00E9444
:1022C00030120CED17E0C80140E052EC61E070E024
:1022D0000E946113C8010E9442140E94550E0E9480
:1022E000F3081F910F910895823000F5E82FF0E078
:1022F000EE0FFF1FE053F94F71836083882319F0BD
:102300008130A1F408C0809169008C7F842B809378
:102310006900E89A089580916900440F551F440FA1
:10232000551F837F842B80936900E99A08951F923B
:102330000F920FB60F9211242F933F934F935F93F9
:102340006F937F938F939F93AF93BF93EF93FF937D
:102350008091D0069091D106892B29F0E091D0068A
:10236000F091D1060995FF91EF91BF91AF919F91A7
:102370008F917F916F915F914F913F912F910F902E
:102380000FBE0F901F9018951F920F920FB60F92CD
:1023900011242F933F934F935F936F937F938F936A
:1023A0009F93AF93BF93EF93FF938091D206909149
:1023B000D306892B29F0E091D206F091D306099536
:1023C000FF91EF91BF91AF919F918F917F916F910D
:1023D0005F914F913F912F910F900FBE0F901F90E3
:1023E0001895CF93DF93482F50E0CA0186569D4F32
:1023F000FC0134914A575D4FFA018491882369F1B9
:1024000090E0880F991FFC01E859FD4FA591B49108
:10241000FC01EE58FD4FC591D491662351F42FB7BE
:10242000F8948C91932F909589238C93888189239C
:102430000BC0623061F42FB7F8948C91932F909574
:1024400089238C938881832B88832FBF06C09FB7F5
:10245000F8948C91832B8C939FBFDF91CF9108953B
:10246000482F50E0CA0182559D4FFC012491CA01BA
:1024700086569D4FFC0194914A575D4FFA01349165
:10248000332309F440C0222351F1233071F024306A
:1024900028F42130A1F0223011F514C02630B1F01B
:1024A0002730C1F02430D9F404C0809180008F77A8
:1024B00003C0809180008F7D8093800010C084B520
:1024C0008F7702C084B58F7D84BD09C08091B00034
:1024D0008F7703C08091B0008F7D8093B000E32F91
:1024E000F0E0EE0FFF1FEE58FD4FA591B4912FB70E
:1024F000F894662321F48C919095892302C08C91E5
:10250000892B8C932FBF0895682F70E0CB018255E3
:102510009D4FFC012491CB0186569D4FFC014491B7
:102520006A577D4FFB019491992319F420E030E024
:102530003CC0222351F1233071F0243028F42130A3
:10254000A1F0223011F514C02630B1F02730C1F0CF
:102550002430D9F404C0809180008F7703C080912B
:1025600080008F7D8093800010C084B58F7702C07B
:1025700084B58F7D84BD09C08091B0008F7703C082
:102580008091B0008F7D8093B000892F90E0880FFC
:10259000991F84589D4FFC01A591B4918C9120E026
:1025A00030E0842311F021E030E0C901089508955E
:1025B0001F920F920FB60F9211242F933F934F93B8
:1025C0008F939F93EF93FF938091C00082FD1DC076
:1025D0004091C60020915407309155072F5F3F4F1F
:1025E0002F77307080915607909157072817390739
:1025F00071F0E0915407F0915507EC52F94F408388
:10260000309355072093540702C08091C600FF9174
:10261000EF919F918F914F913F912F910F900FBE0E
:102620000F901F901895E091E807F091E907E058A6
:10263000FF4F8191919120813181821B930B8F7784
:102640009070892B11F00E94D71208951F920F925B
:102650000FB60F9211242F933F938F939F93EF9375
:10266000FF932091D8073091D9078091DA07909194
:10267000DB072817390731F48091C1008F7D8093E3
:10268000C10014C0E091DA07F091DB07E85AF84F77
:1026900020818091DA079091DB0701968F77907007
:1026A0009093DB078093DA072093C600FF91EF91A8
:1026B0009F918F913F912F910F900FBE0F901F9080
:1026C0001895AF92BF92DF92EF92FF920F931F93F4
:1026D000CF93DF93EC017A018B01DD24403081EE52
:1026E000580780E0680780E0780711F0DD24D39474
:1026F00091E0A92EB12CEC89FD89DD2069F0C5019E
:1027000008A002C0880F991F0A94E2F7808360E056
:1027100079E08DE390E005C0108260E874E88EE116
:1027200090E0A80197010E94B71521503040404029
:102730005040569547953795279580E120303807CA
:1027400020F0DD2011F0DD24D6CFE889F98930832F
:10275000EA89FB89208319A2EE89FF89408121E063
:1027600030E0C9010C8C02C0880F991F0A94E2F76F
:10277000482B4083EE89FF894081C9010D8C02C03E
:10278000880F991F0A94E2F7482B4083EE89FF894E
:102790004081C9010E8C02C0880F991F0A94E2F78C
:1027A000482B4083EE89FF8980810F8C02C0220F65
:1027B000331F0A94E2F7209528232083DF91CF91DD
:1027C0001F910F91FF90EF90DF90BF90AF90089511
:1027D000DC011C96ED91FC911D97E058FF4F219173
:1027E000319180819181281B390B2F773070C9017D
:1027F0000895DC011C96ED91FC911D97E058FF4F68
:1028000020813181E058F040DF01AE57BF4F8D91FC
:102810009C9111972817390719F42FEF3FEF07C044
:102820008D919C91E80FF91F8081282F30E0C9011C
:102830000895DC011C96ED91FC911D97E058FF4F27
:1028400020813181E058F040DF01AE57BF4F8D91BC
:102850009C9111972817390719F42FEF3FEF10C0FB
:102860008D919C911197E80FF91F20818D919C917A
:10287000119701968F77907011969C938E9330E00C
:10288000C9010895DC0191968C919197882339F0C4
:102890005496ED91FC915597808186FFF9CF9196E2
:1028A0001C920895CF93DF93EC01EE85FF85E058ED
:1028B000FF4F20813181E058F0402F5F3F4F2F774D
:1028C0003070DF01AE57BF4F8D919C911197281743
:1028D0003907D1F3E058FF4F80819181E058F040F3
:1028E000E80FF91F6083EE85FF85E058FF4F3183C5
:1028F0002083EE89FF89208181E090E00F8C02C067
:10290000880F991F0A94E2F7282B208381E089A37E
:10291000EC89FD8980818064808381E090E0DF9193
:10292000CF9108951092DF071092DE0788EE93E0B2
:10293000A0E0B0E08093E0079093E107A093E20766
:10294000B093E30789E091E09093DD078093DC0783
:1029500084ED96E09093E9078093E80788E597E097
:102960009093EB078093EA0785EC90E09093ED0756
:102970008093EC0784EC90E09093EF078093EE0750
:1029800080EC90E09093F1078093F00781EC90E069
:102990009093F3078093F20782EC90E09093F50711
:1029A0008093F40786EC90E09093F7078093F60706
:1029B00084E08093F80783E08093F90787E08093B1
:1029C000FA0785E08093FB0781E08093FC07089578
:1029D000CF93DF930E9469150E943711C3E1D3E1C1
:1029E0000E94810E2097E1F30E941313F9CFCF923A
:1029F000DF92EF92FF920F931F93CF93DF937C01AF
:102A00006B018A01C0E0D0E00FC0D6016D916D016D
:102A1000D701ED91FC910190F081E02DC70109955E
:102A2000C80FD91F015010400115110571F7CE01D3
:102A3000DF91CF911F910F91FF90EF90DF90CF909A
:102A400008951F920F920FB60F9211242F933F9368
:102A50008F939F93AF93BF93809102089091030847
:102A6000A0910408B0910508309106080196A11DB7
:102A7000B11D232F2D5F2D3720F02D570196A11D5D
:102A8000B11D209306088093020890930308A09339
:102A90000408B09305088091FE079091FF07A0916C
:102AA0000008B09101080196A11DB11D8093FE0799
:102AB0009093FF07A0930008B0930108BF91AF91D6
:102AC0009F918F913F912F910F900FBE0F901F906C
:102AD0001895789484B5826084BD84B5816084BD86
:102AE00085B5826085BD85B5816085BDEEE6F0E087
:102AF000808181608083E1E8F0E0108280818260E3
:102B00008083808181608083E0E8F0E08081816063
:102B10008083E1EBF0E0808184608083E0EBF0E093
:102B2000808181608083EAE7F0E080818460808337
:102B300080818260808380818160808380818068E1
:102B400080831092C100089597FB092E07260AD0B2
:102B500077FD04D02ED006D000201AF47095619530
:102B60007F4F0895F6F7909581959F4F0895A1E2C4
:102B70001A2EAA1BBB1BFD010DC0AA1FBB1FEE1FF7
:102B8000FF1FA217B307E407F50720F0A21BB30B42
:102B9000E40BF50B661F771F881F991F1A9469F7BE
:102BA00060957095809590959B01AC01BD01CF011A
:102BB0000895AA1BBB1B51E107C0AA1FBB1FA61784
:102BC000B70710F0A61BB70B881F991F5A95A9F7D6
:102BD00080959095BC01CD010895EE0FFF1F0590E3
:0A2BE000F491E02D0994F894FFCF62
:102BEA002C01FA0001000000005214F714E813192E
:062BFA0014F9134214005F
:00000001FF
